:1000000016EF00F0EA6A060EE96EEF500EE0010E00
:10001000016E006A002EFED7012EFBD74A0E006E3D
:10002000002EFED700D0EF2EF2D7000CF86AD09E3B
:10003000EA6AE96A600ED36ED350C150C00B0F0953
:10004000C16E070EB46EC150C00B0F09C16EC090D7
:10005000C092C094C09EC280B098C69A949A948868
:100060009496010EC66E000EC76ED190800ED56EAE
:10007000CD6A000ECA6E000ECB6E9484BD6A070E68
:10008000B46E9750976E030E006E002EFED7B450DC
:10009000A19CB56A9A9C919C040E056EFA0E066EA0
:1000A000B1DF052EFBD79A9C918C040E056EFA0EDB
:0C00B000066EA8DF052EFBD7EDD703007D
:020000040030CA
:0E0000000088190EC385810001000000010078
:00000001FF
